:060000000A128A11122809
:10000800FE00030EF1000408F2000A08F300831250
:1000180003137F08F4000A128A11FB2B0A128A11B3
:100028001528F501F601F701F80183120313C6013B
:100038008313A0308400F0300A128A112D24830122
:100048000A128A112728073083120313C1004108B6
:10005800831603139F049F111F159F141F148030CC
:100068008700FF308500831203138512831603135C
:10007800880183120313081288118812881000302F
:10008800B2000030B1002530B0008030AF000A1255
:100098008A11E7210A128A11153083120313C3004B
:1000A8004B30C200BD30C100C10B5828C20B5828C4
:1000B800C30B58285F288312031308129930831240
:1000C8000313C3003130C200A130C100C10B6A283C
:1000D800C20B6A28C30B6A2871286C300A128A116D
:1000E800D5230A128A110D300A128A1121240A1204
:1000F8008A11063083120313C3001330C200AD30D7
:10010800C100C10B8528C20B8528C30B85286C301C
:100118000A128A11D5230A128A110D300A128A117D
:1001280021240A128A11063083120313C3001330E4
:10013800C200AD30C100C10B9F28C20B9F28C30B62
:100148009F2867300A128A11D5230A128A110D30A6
:100158000A128A1121240A128A1106308312031303
:10016800C3001330C200AD30C100C10BB928C20BA7
:10017800B928C30BB9283A300A128A11D5230A12B2
:100188008A110D300A128A1121240A128A110630A6
:1001980083120313C3001330C200AD30C100C10B7A
:1001A800D328C20BD328C30BD3281C300A128A11B8
:1001B800D5230A128A110D300A128A1121240A1233
:1001C8008A110B3083120313C3002630C2005D303E
:1001D800C100C10BED28C20BED28C30BED2844303C
:1001E8000A128A11D5230A128A1122300A128A1198
:1001F80021240A128A1157300A128A11D5230A12A9
:100208008A1122300A128A1121240A128A110D3009
:100218000A128A1121240A128A110B30831203133D
:10022800C3002630C2005D30C100C10B1929C20BC2
:100238001929C30B19294E300A128A11D5230A121B
:100248008A1122300A128A1121240A128A112E30A8
:100258000A128A11D5230A128A1122300A128A1127
:1002680021240A128A110D300A128A1121240A1235
:100278008A110B3083120313C3002630C2005D308D
:10028800C100C10B4529C20B4529C30B45290130C3
:100298000A128A11D5230A128A110D300A128A11FC
:1002A80021240A128A111A300A128A1121240A12E8
:1002B8008A11333083120313C300BB30C200DF300E
:1002C800C100C10B6529C20B6529C30B65293330F1
:1002D80083120313C300BB30C200DF30C100C10B5F
:1002E8007329C20B7329C30B7329831203138C124E
:1002F800C401C5018B170B17831603138C168312C1
:1003080003134603031D7E293A300A128A11D523A6
:100318000A128A110D300A128A1121240A128A112E
:10032800063083120313C3001330C200AD30C1007E
:10033800C10B9C29C20B9C29C30B9C294E300A1265
:100348008A11D5230A128A1122300A128A1121240D
:100358000A128A112E300A128A11D5230A128A111A
:1003680022300A128A1121240A128A110D300A1227
:100378008A1121240A128A110B3083120313C30035
:100388002630C2005D30C100C10BC829C20BC82984
:10039800C30BC8295F300A128A11D5230A128A11A1
:1003A8000D300A128A1121240A128A111A300A12EF
:1003B8008A1121240A128A11023083120313C10000
:1003C8004108C6007E29831203132F08B3003008A2
:1003D800B4003108B5003208B60006300310B30D7A
:1003E800B40DB50DB60DFF3E031DF2293608A30066
:1003F8003508A2003408A1003308A0000030B70077
:100408001230B8007A30B9000030BA002F08BB00AB
:100418003008BC003108BD003208BE0006300310A9
:10042800BB0DBC0DBD0DBE0DFF3E031D132ABB0940
:10043800BC09BD09BE09BB0A0319BC0A0319BD0AD8
:100448000319BE0A3B08B7073C0803183C0F2D2ABE
:100458002E2AB8073D0803183D0F332A342AB90756
:100468003E0803183E0ABA073A08A7003908A6004A
:100478003808A5003708A4000A128A11D2220A12E5
:100488008A11831203132108C0002008BF0001301D
:100498004002003003193F02031CB72A2F08B3009B
:1004A8003008B4003108B5003208B6000430031033
:1004B800B30DB40DB50DB60DFF3E031D5B2A36080E
:1004C800A3003508A2003408A1003308A0000030BA
:1004D800B7001230B8007A30B9000030BA002F08DF
:1004E800BB003008BC003108BD003208BE00043033
:1004F8000310BB0DBC0DBD0DBE0DFF3E031D7C2AB8
:10050800BB09BC09BD09BE09BB0A0319BC0A03190A
:10051800BD0A0319BE0A3B08B7073C0803183C0F7D
:10052800962A972AB8073D0803183D0F9C2A9D2A4A
:10053800B9073E0803183E0ABA073A08A70039085F
:10054800A6003808A5003708A4000A128A11D2228A
:100558000A128A11831203132108C0002008BF0061
:100568008316031318150130831240020030031953
:100578003F02031808003F08831603139900181256
:10058800831203139817803083160313870083128E
:1005980003131816831603139816080083120313FF
:1005A800AA01A31FE42AA009A109A209A309A00A74
:1005B8000319A10A0319A20A0319A30AAA01AA0A7C
:1005C800A71FF52AA409A509A609A709A40A0319BA
:1005D800A50A0319A60A0319A70A0130A8002808C2
:1005E800AA060030AE000030AD000030AC0000308C
:1005F800AB00230822042104200403194A2BA90173
:10060800A90AA31B152B0130A8000310A00DA10DEA
:10061800A20DA30DA80B092B0130A8002808A907D3
:10062800052B0130A8000310AB0DAC0DAD0DAE0DC0
:10063800A80B172B23082702031D2C2B22082602A0
:10064800031D2C2B21082502031D2C2B2008240216
:10065800031C3D2B2008A4022108031C210FA5021E
:100668002208031C220FA6022308031C230FA7023B
:100678002B1401300310A30CA20CA10CA00CFF3EFC
:10068800031D3E2B0130A902031D152B2A0803194F
:10069800582BAB09AC09AD09AE09AB0A0319AC0A72
:1006A8000319AD0A0319AE0A2E08A3002D08A200EB
:1006B8002C08A1002B08A000080003308A000408B9
:1006C800840A82070034483465342034743468342A
:1006D8006F346E34673420346434613420346434C5
:1006E80075346F34633420346B3468346F34693450
:1006F800203464346F346E346734003441345434F5
:100708002B3443344E344D3449343D3432342C3454
:1007180032342C3430342C3430342C3430340034EB
:100728003034313436343334353435343034363487
:100738003234383439340034413454342B3443346B
:100748004D34473446343D34313400344134543424
:100758002B3443344D344734443441343D3400342D
:10076800413454342B3443344D34473453343D34BA
:100778000034443445344C34203441344C344C3403
:1007880000346434613420346E34683461346E3437
:100798000034413454344534303400344134543412
:1007A800003483120313A300A101A2012108230727
:1007B80084000A128A1161230A128A11003A031965
:1007C80008002108230784000A128A1161230A12EB
:1007D8008A110A128A1121240A128A1101308312FD
:1007E8000313A1070318A20A0030A207DA2B8C1EF4
:1007F800162C0130F0007008C6001A08F0007708BF
:10080800A03E84007008831380000130F7070318A6
:10081800F80A0030F807981C162C181200008312EA
:10082800031318167408FF0073088A0072088400FE
:10083800710E8300FE0E7E0E090083120313A000C2
:1008480083160313981C242C831203132008990081
:10085800080064008001840A0406031900340406B1
:020868002E2C34
:02400E003A3F37
:00000001FF
